:020000040000FA
:040000000B303A285F
:08000800A000030EA100831209
:100010008B1C32288B1031181428B11C3228643004
:10002000010203183128182800001628172818285C
:1000300019281A281B281C281D281E281F283110A3
:10004000B114A810031005190314AA0DA90DA80DC9
:10005000B00B322831152A08AF002908AE00280855
:10006000AD00B11081010B11210E8300A00E200EF6
:02007000090085
:0C007400203084008001840A6030040207
:10008000031C3C281230B0002C228316FF23900062
:1000900083128316851683120C30851A2C30831632
:1000A000850083128501870107309900003083168F
:1000B00091009F008312C830831681008312313073
:1000C0009000003083168C00831210308B00831652
:1000D00000309B001C141A088312BC00851DA82246
:1000E0003C1C7A28831610309B001C141A088312BB
:1000F000BD007422831620309B001C141A08831242
:10010000C1000130C1080319C10081018E018F01B6
:100110000B118B100B108C018B179D203119B32004
:100120001022B30B9B28031085190314B90DF0306E
:1001300039020319A2217D228D286400311808009C
:100140000B1D08000B11B11031141230B000051D49
:10015000AE2832148316011383120800321083165E
:1001600001178312080031110130B7008B132030C2
:10017000370783169B001C141A088312A400A500DD
:10018000C030A5061030370783169B001C141A08D0
:100190008312A3000030370783169B001C141A0833
:1001A0008312A2008B17321CDB2822090339A2001C
:1001B000A309A409A50922082D02031D9C292308CF
:1001C0002E02031D9C2924082F02031D3F29013004
:1001D0003702031DF2283C19F1283D18F2283D147E
:1001E0003E142D2202303702031DFD283C19FC2845
:1001F000BD18FD28BD143E14342203303702031D00
:1002000008293C1907293D1908293D153E143B22B0
:1002100004303702031D13293C191229BD19132973
:10022000BD153E14422205303702031D1E293C191C
:100230001D293D1A1E293D163E144922063037025B
:10024000031D29293C192829BD1A2929BD163E1448
:100250004A2207303702031D34293C1933293D1B3C
:1002600034293D173E144B2208303702031D3F2925
:100270003C193E29BD1B3F29BD173E144C222508C1
:100280002F02031D9C2901303702031D4E293C1902
:100290004D293D1C4E293D103E144D22023037029F
:1002A000031D59293C195829BD1C5929BD103E145C
:1002B0004F2203303702031D64293C1963293D1D79
:1002C00064293D113E14512204303702031D6F2969
:1002D0003C196E29BD1D6F29BD113E1453220530F6
:1002E0003702031D7A293C1979293D1E7A293D12CE
:1002F0003E145A2206303702031D85293C198429F1
:10030000BD1E8529BD123E145B2207303702031D36
:1003100090293C198F293D1F90293D133E145C22E2
:1003200008303702031D9B293C199A29BD1F9B29C0
:10033000BD133E145D229C29B70A0530370203180D
:100340000800B6280130B600B300B400B500B7000D
:1003500004308316851AB700831285018701B11313
:100360009D20B30BDF29031085190314B90DF0305C
:1003700039020319062AB40BDF29013037020319A9
:100380005E2202303702031962220330370203195A
:1003900066220430370203196A2205303702031936
:1003A0006E220630370203196F2207303702031915
:1003B000702208303702031971229630B400311DC3
:1003C000B0293111321CE9292D090339AD00AE09DC
:1003D000AF092F1CB1132F1CB029B11BB0292E1847
:1003E000B029B1178B1320303707BB002F08BA0094
:1003F000192210303707BB002E08BA00192200302E
:100400003707BB002D08BA0019228B178501870119
:10041000B70AB60105303702031CB0297422080060
:100420003E1C08003E101030BB003D08BA001922E7
:1004300008008B133A0883161C159A003B089B0092
:1004400055309D00AA309D009C1464009C18252AFC
:100450001C1183128B1708000800851440084107FF
:10046000D0000F08D1000800051440084107D20051
:100470000F08D3000800851640084107D4000F0874
:10048000D5000800051640084107D6000F08D70020
:100490000800080008000800080085100800051082
:1004A00008008512080005128E018F010C1041080A
:1004B000C000080008000800080008000508023A0B
:1004C000850008000508013A850008000508203A63
:1004D000850008000508103A85000800080008009B
:1004E00008000800080008003D188514BD18051410
:1004F0003D198516BD19051608003C1D0800500859
:100500004002031D882A51080F02031C882A851007
:1005100052084002031D912A53080F02031C912A1E
:10052000051054084002031D9A2A55080F02031CA7
:100530009A2A851256084002031DA32A57080F0263
:10054000031CA32A05120C1C08000C10C00A08008A
:10055000B601B301B4013C1CB02ABC01BC14B72ADB
:10056000BC1CB52ABC013C15B72ABC013C143C0894
:10057000B6006400BB2ABC2ABD2ABE2ABF2AB41B0F
:100580008514B41F8510B30BB92AB40BB92A031014
:10059000B60CB608031DB92A0030BB003C08BA00EF
:0405A0001922080014
:084000000D000300030009009C
:02400E00CC01E3
:10420000010003000300030003000200020002009B
:1042100002000000000000000000FF00FF00FF009F
:10422000000000000000000000000000000000008E
:104230000000C000C000C000C000FF00FF00FF0081
:104240000100C300F300CF00FF00C300F300CF0064
:10425000FF00C300F300CF00FF00FF00FF00FF00DE
:10426000FF00FF00FF00FF00FF00FF00FF00FF0056
:10427000FF00FF00FF00FF00FF00FF00FF00FF0046
:10428000FF00FF00FF00FF00FF00FF00FF00FF0036
:10429000FF00FF00FF00FF00FF00FF00FF00FF0026
:1042A000FF00FF00FF00FF00FF00FF00FF00FF0016
:1042B000FF00FF00FF00FF00FF00FF00FF00FF0006
:1042C000FF00FF00FF00FF00FF00FF00FF00FF00F6
:1042D000FF00FF00FF00FF00FF00FF00FF00FF00E6
:1042E000FF00FF00FF00FF00FF00FF00FF00FF00D6
:1042F000FF00FF00FF00FF00FF00FF00FF00AA001B
:00000001FF
